S01B00006F70656E62746C5F656B5F6C6D3373383936322E737265632F
S1130000E8050020B90B0000ED190000ED1900000F
S1130010ED190000ED190000ED190000ED190000C4
S1130020ED190000ED190000ED190000ED190000B4
S1130030ED190000ED190000ED190000ED190000A4
S1130040ED190000ED190000ED190000ED19000094
S1130050ED190000ED190000ED190000ED19000084
S1130060ED190000ED190000ED190000ED19000074
S1130070ED190000ED190000ED190000ED19000064
S1130080ED190000ED190000ED190000ED19000054
S1130090ED190000ED190000ED190000ED19000044
S11300A0ED190000ED190000ED190000ED19000034
S11300B0ED190000ED190000ED190000ED19000024
S11300C0ED190000ED190000ED190000ED19000014
S11300D0ED190000ED190000ED190000ED19000004
S11300E0ED190000ED190000ED190000ED190000F4
S11300F0044B9D46C046C046C046C04600F08DFC39
S113010000F0F8FFE8050020DFF86C14884200F0E6
S1130110A980DFF86814884200F0A480DFF8601436
S1130120884200F09F80DFF85C14884200F09A80D7
S1130130DFF85414884200F09580DFF850148842A8
S113014000F09080DFF84814884200F08B80DFF8DC
S11301504414884200F08680DFF83C14884200F0A2
S11301608180DFF8381488427CD0DFF83414884268
S113017078D0DFF83014884274D0DFF82C14884229
S113018070D0DFF8281488426CD0DFF82414884239
S113019068D0DFF82014884264D0DFF81C14884249
S11301A060D0DFF8181488425CD0DFF81414884259
S11301B058D0402856D0B0F1102F53D0DFF8041493
S11301C088424FD0DFF8001488424BD0DFF8FC138C
S11301D0884247D0DFF8F813884243D0DFF8F4139D
S11301E088423FD0B0F1101F3CD0DFF8EC138842B6
S11301F038D0DFF8E813884234D0DFF8E4138842BB
S113020030D0DFF8E01388422CD0DFF8DC138842CA
S113021028D0DFF8D813884224D0DFF8D4138842DA
S113022020D0DFF8D01388421CD0DFF8CC138842EA
S113023018D0DFF8C813884214D0DFF8C4138842FA
S113024010D0DFF8C01388420CD0B0F1202F09D0B1
S1130250DFF8B413884205D0082803D0DFF8AC13C4
S1130260884201D1012070470020704738B5044608
S1130270DFF89C53FFF748FF002805D14FF4FC71C9
S113028005F19C0000F0E8F9200F05EB8000C0693F
S11302900168A2B2230C03F01F039A4011430160CA
S11302A031BD00000138FDD170477047F8B50446F0
S11302B0DFF86053286810F0E04F06D02868DFF8B4
S11302C058130840B0F1805F01D1002C7DD4286E12
S11302D0296F20F4800040F4006641F400672E6624
S11302E02F673046800702D52046800707D506F0E1
S11302F0010004F0010181F0010108421AD064F008
S1130300030006402E66002F05D507F07000302844
S113031007D0702805D0002F08D406F0300030280C
S113032004D14FF48050FFF7BDFF03E04FF40020E9
S1130330FFF7B8FFDFF8E402304043F2F0712140E8
S113034041EA0006DFF8D8023840DFF8D81221402D
S1130350084304F0080140EAC1074020A865002FC3
S113036002D52F672E6601E02E662F671020FFF757
S113037099FFDFF8B4023040DFF8B012214008439F
S1130380E10D61F3DC57610008D540F4800027F4E7
S11303908001DFF89C222240114301E027F08041D4
S11303A022050CD44FF4004200E0521E002A02D071
S11303B02B6D5B06F9D520F4006021F400612866FA
S11303C029671020BDE8F2406CE7F1BD70B4DFF896
S11303D044120A6E0B6F002B02D503F0700001E08B
S11303E002F0300000280DD0102835D020285BD032
S11303F0302800F08180602800F08180702800F0AF
S1130400818082E0C2F38410DFF8044204EB8000B0
S1130410006CDFF8204204EA030515F1004F05D013
S1130420002B00F18580150500F182804D6E0E6869
S113043016F0E04F06D00968DFF8DC613140B1F115
S1130440805F64D1C5F34811891C484305F01F013E
S1130450891CB0FBF1F063E0086810F0E04F06D0AF
S1130460DFF8B4010C680440B4F1805F02D1DFF816
S1130470C801CEE70C680440DFF8C051AC4203D198
S11304800C68A4B2022C09D00C682040DFF8B041FB
S1130490A04206D1086880B2002802D1DFF8A40186
S11304A0B7E7DFF8A401B4E7086810F0E04F06D01E
S11304B0DFF864010C680440B4F1805F02D1DFF816
S11304C08C01A6E70C680440DFF87051AC4203D1FC
S11304D00C68A4B2022C09D00C682040DFF86041FB
S11304E0A04206D1086880B2002802D1DFF860017A
S11304F08FE7DFF860018CE747F2305089E74FF46B
S1130500800086E74FF4004083E7002031E0C5F324
S11305104811484305F01F01491C4900B0FBF1F0A4
S1130520690400D54008290400D5800842F48002FB
S113053051021ED5002B17D559000FD504EA03012B
S113054011F1004F03D0002B08D4110506D440004C
S1130550C3F38651491CB0FBF1F00AE0C3F3C55163
S1130560491CB0FBF1F004E0C2F3C351491CB0FBD9
S1130570F1F070BC70470000010010000200100090
S1130580000110000002100000041000000110100F
S11305900002101000041010004010100050102031
S11305A001000020020000200400002008000020B8
S11305B010000020200000204000002080000020C7
S11305C00001002000400010001010100001102055
S11305D08000003010000030000100100002001004
S11305E01000001020000010200000300100101046
S11305F00200101004001010080010100100001078
S1130600020000100400001001001020001010006F
S1130610D815000000E00F400000FF700FC8FFFF76
S11306208FDFFF7F30200080FCFF3FF80300C0070E
S11306300000404000080080C0E1E4000000011018
S113064000000310001BB7000024F40070383900C8
S1130650C0C62D0000093D0080B5034A10605160FA
S113066000F005F8FCE700BFDC0400207047704789
S1130670D34800210180816480F84310A0F844101D
S113068081707047CE480178481E8041C043C00F36
S11306907047CB48002180F84310704710B5C84C10
S11306A00178FF2902D100F07EF84DE0217801297C
S11306B05AD10178C92932D0CC293FD0CF293AD098
S11306C0D0292FD0D12933D0D2292ED0F32917D035
S11306D0F4290FD0F5290AD0F6290ED0FA2912D020
S11306E0FC2913D0FD2914D0FE2915D029E000F0EF
S11306F0AAF829E000F0C2F826E000F09BF823E015
S113070000F0D9F820E000F084F81DE000F07FF854
S11307101AE000F06CF817E000F05DF814E000F067
S1130720EFF811E000F004F90EE000F0D7F80BE068
S113073000F029F908E000F038F905E000F044F988
S113074002E0202000F027F894F84300012802D1A9
S1130750102000F020F8012084F84300B4F944107C
S1130760E01CBDE8104000E010BD89B200F04DB9B6
S113077010B4002303E00478E318DBB2401C0C46F9
S1130780611E002CF7D11360012010BC70478C4807
S11307900021417070478A49FE22CA700871022004
S11307A0A1F84400704780B5FFF7F1FF84480121A8
S11307B00170FF21C170102101710021417140219C
S11307C08171C1710021017201214172817208217C
S11307D0A0F8441001BD10B5794C00202070FFF73B
S11307E0D6FFFF20E0700120A4F8440010BD744837
S11307F0411CFF228A700022CA7042780A710022CA
S11308004A718A71CA710621A0F844107047002009
S1130810C1E76B48FF21C1706A49816400F203019A
S113082000224A708A70CA7007224A600821A0F820
S1130830441070476249FF22CA70406888640120EE
S1130840A1F84400704770B505466A78402A03D37E
S11308502220BDE870409EE7594C04F244067168BA
S1130860201D00F0FFF8FF20E07070686978081818
S113087070606878401CA4F8440070BD70B50546EB
S11308806878402803D32220BDE8704083E7696874
S11308904B4C04F2440671606A78201D00F0E2F8C3
S11308A0FF20E07070686978081870606878401CF0
S11308B0A4F8440070BD38B5414CFF21E17004F246
S11308C00305E21D4168A06CFFF752FF6870002029
S11308D0A870E8700820A4F8440031BD3848FF210E
S11308E0C17000F2030100224A708A704022CA706B
S11308F000220A714A718A710721A0F844107047D6
S113090038B52F4C04F24405421C3F21686800F0BE
S1130910BEF8002803D13120BDE832403BE7FF2078
S1130920E07068683F3068600120A4F8440031BD7D
S113093038B5044660783F2803D32220BDE832400E
S113094029E71F48FF21C1700121A0F844106178F4
S1130950002907D100F0A1F8002813D13120BDE807
S1130960324018E700F24405A21C686800F08FF8D2
S1130970002803D13120BDE832400CE76868617873
S11309800818686031BD10B50D4C4168A06C00F0CA
S113099080F8002803D13120BDE81040FBE6FF2099
S11309A0E0700120A4F8440010BD80B500F06BF89D
S11309B00348FF21C1700121A0F8441001BD0000CB
S11309C008040020041A00003120E4E680B500A8E1
S11309D016490A880280FFF74BFE00F069F81448B4
S11309E00078012802D100A8FFF758FE01BD10B518
S11309F0104C204600F090F8012804D12046BDE8B0
S1130A001040FFF74BBE10BD704780B5C9B200F06F
S1130A105EF8BDE80140FFF73CBE054801210170C6
S1130A207047034800210170704700002E15000034
S1130A30E80500209C040020FFF724BE80B500F0E8
S1130A402AF800280BD0FFF7DFFF05484FF40051C8
S1130A50016042F204000068BDE80240004701BDA5
S1130A6008ED00E070B504460D46164605E015F89D
S1130A70010B04F8010BFFF7FAFD3046461E80B265
S1130A800028F4D170BD00F097B800F0A1B800F0D0
S1130A90A6B800F0C5B800F0F7B880B500F0D5F8F6
S1130AA0002801D1002002BDBDE8014000F003B9D7
S1130AB080B53D48FFF7DAFBFFF788FC60234FF46D
S1130AC0614201463948BDE8005000F029BA70B5CA
S1130AD004460D46412D03D357213548FFF7BCFD8D
S1130AE0284600F04EF8012803D05A213048FFF779
S1130AF0B3FD00260BE0FFF7BAFD305D00F041F8CE
S1130B00012803D062212A48FFF7A6FD761C284657
S1130B10B6B28642EFD370BD38B50546254C607831
S1130B2000280AD1201D00F01FF8012803D101205C
S1130B30607000202070002032BD20780019401D14
S1130B4000F012F80128F6D12078421C2270207996
S1130B50D2B28242EFD1201D411C2846FFF782FF0A
S1130B6000206070012032BD10B504460F4800F02B
S1130B7087FA10F1010F02D02070012010BD00206F
S1130B8010BD10B5094C0146204600F08CFA00282F
S1130B9003D1002010BDFFF76AFD204600F05DFA86
S1130BA00028F8D0012010BD0100001000C0004052
S1130BB09C19000054040020044B9D46C046C046C6
S1130BC0C046C046FFF72DFF00F094FAE805002068
S1130BD04FF0FF30C7490860C7490860704770B5D7
S1130BE004460D46164600F03EF9FF2805D02819A4
S1130BF0401E00F038F9FF2801D1002070BD600AC2
S1130C004002B0F5005F2B469BB23246214603D129
S1130C10B948BDE8704094E0B648BDE8704090E043
S1130C2070B504460D4600F01EF906462819401E0C
S1130C3000F019F9FF2E01D0FF2801D1002070BD6A
S1130C4001463046BDE87040E2E080B5AA4801683C
S1130C5011F1010F01D1012002BD416882685118D0
S1130C60C2685118026951184269511882695118B1
S1130C70C0694018C043401C009000AA042142F2FD
S1130C80F000FFF7ACFF02BD4FF40050016842686A
S1130C90511882685118C268511802695118426982
S1130CA051188069401842F2F00109680818401E82
S1130CB08041C00F704780B58F48016811F1010F62
S1130CC003D000F07FF8002808D08A48016811F1A9
S1130CD0010F05D000F076F8002801D1002002BDF4
S1130CE0012002BD80B5CA0501D0002002BD026802
S1130CF08A4201D1012002BD01604FF40072001D3F
S1130D00FFF7B0FE012002BD38B504460D467A480F
S1130D10844208D1774C29462046FFF7E3FF002898
S1130D200DD1002032BDB5F5005F01D10446F2E7D4
S1130D30204600F047F80028EDD1002032BD2046BF
S1130D4032BD2DE9F0410746884614461D464FEA58
S1130D5058267602386810F1010F05D1314638461D
S1130D60FFF7C0FF00281ED03868B04205D03146D6
S1130D703846FFF7C9FF070015D03868A8EB000014
S1130D80C01900F10408FFF772FC381DA8EB00003D
S1130D904FF4007188420AD306F200213846FFF767
S1130DA0B3FF070001D100200AE007F1040814F89A
S1130DB0010B08F8010B6D1EADB2002DE3D101202B
S1130DC0BDE8F081F8B504460125206800F04BF831
S1130DD0FF2801D10020F2BD002600E0761C802E01
S1130DE014D2216811EB860714EB8600406800904A
S1130DF0FFF73DFC0422394600A800F0B3F90028AF
S1130E0003D1386800998842E8D000252846F2BD0D
S1130E10F8B50D46854222D3002820D0142D1ED2C9
S1130E2000F03BF80446284600F037F8064628460A
S1130E3000F04AF88019401E001B401C850AADB220
S1130E40002600E0761CB6B23746AF4209DAFFF757
S1130E500EFC04EB872000F069F90028F2D0002092
S1130E60F2BD0120F2BD38B50446002501E06D1C39
S1130E70EDB2132D0FD2FFF7FAFB05EB450080000E
S1130E801E4942589442F2D34018416889188C4252
S1130E90EDD2007A32BDFF2032BD38B504460025BC
S1130EA000E06D1CEDB2132D0BD2FFF7E0FB05EB58
S1130EB04500800011494218127AA242F1D14058EB
S1130EC032BD4FF0FF3032BD38B50446002500E096
S1130ED06D1CEDB2132D0BD2FFF7C9FB05EB4500DA
S1130EE0064901EB8000017AA142F1D1406832BD8C
S1130EF0002032BD0000002004020020D8160000AB
S1130F00DFF8CC11884207D0DFF8C811884203D03B
S1130F10DFF8C411884201D10120704700207047D6
S1130F20F8B504460E4617461D46FFF7E9FF0028AC
S1130F3005D140F20D11DFF8A401FFF78DFB002F5E
S1130F4005D14FF48771DFF89401FFF785FBDFF8D3
S1130F509001016811F0E04F1AD0DFF8881102689F
S1130F600A40B2F1805F13D002680A40DFF878319A
S1130F709A4203D1026892B2022A09D0026811404F
S1130F80DFF86821914205D1006880B2002801D1C0
S1130F90102000E008207843864205D240F20F1169
S1130FA0DFF83801FFF758FB204600F039F804F168
S1130FB03000B6EB071F016804D241F02001016044
S1130FC07F0802E021F020010160F000B0FBF7F09F
S1130FD0401C40088109616200F03F00A062E562A4
S1130FE00020A0612046BDE8F240FFE710B50446AA
S1130FF0FFF786FF002805D14FF4CF71DFF8DC003E
S1131000FFF72AFB04F12C00016841F01001016094
S113101004F13000016840F201321143016010BD57
S113102010B50446FFF76CFF002805D14FF4DF71BB
S1131030DFF8A800FFF710FBA0690007FCD404F157
S11310402C00016821F01001016004F130000168F6
S1131050DFF89C201140016010BD10B50446FFF775
S11310604FFF002804D140F2E9311C48FFF7F4FA9D
S1131070A069C0B2400900F0010080F0010010BD79
S113108010B50446FFF73CFF002804D140F20941A3
S11310901248FFF7E1FAA069C00601D4206810BD28
S11310A04FF0FF3010BD38B504460D46FFF728FF5A
S11310B0002804D140F25B410848FFF7CDFAA0694B
S11310C0800602D42560012032BD002032BD00001C
S11310D000C0004000D0004000E00040F0180000D4
S11310E000E00F400000FF7000000110000003103A
S11310F0FEFCFFFF00F090F8002801D000F08EF80D
S1131100002000F0A1F800F0B9F850F8041B61B118
S113111050F8042BD30744BFA9F101039A18002304
S113112042F8043B091FFAD1EFE7704710B50446B3
S1131130A00504D08421DFF8C800FFF78DFADFF89A
S1131140C400012141610460DFF8BC108160816842
S11311508907FCD4C068C00702D54FF0FF3010BD2A
S1131160002010BD70B504460D46164615F0030068
S113117004D0C821DFF88800FFF76EFA16F00300E8
S113118004D0C921DFF87800FFF766FADFF87400AD
S113119001214161DFF874100968C90726D5002EC2
S11311A026D0E909C9010160194A06E005F07C016D
S11311B054F8043B53502D1D361F15F07C0102D109
S11311C0016B002901D1002EF0D112490162016A9C
S11311D0C907FCD4E3E70560216841600D498160DB
S11311E08168C907FCD4241D2D1D361F002EF2D1A1
S11311F0C068C00702D54FF0FF3070BD002070BD3D
S11312008818000000D00F40020042A4A0E10F4063
S113121000D10F40010042A40120704710B50849D5
S113122079441C31074C7C441A34A14206D0081D71
S11312300A68511888470146A142F8D110BD00BF81
S11312409C070000A807000080B500F005F800F036
S113125017F800F020F8FCE780B50648FFF726F8F9
S11312600548FFF703F803214FF04020BDE8044090
S113127000F01BB98003C0010100002000F052B946
S113128080B5FFF7F3F900F053F9FFF7FEFBBDE873
S11312900140FFF79BBB80B5FFF7E9F9FFF7A7FB18
S11312A0BDE8014000F04CB9B0F1402F43D0DFF865
S11312B02C1288423FD0DFF8281288423BD0DFF856
S11312C02412884237D0DFF82012884233D0DFF866
S11312D01C1288422FD0DFF8181288422BD0DFF876
S11312E01412884227D0DFF81012884223D0DFF886
S11312F00C1288421FD0DFF8081288421BD0DFF896
S11313000412884217D0DFF80012884213D0DFF8A5
S1131310FC1188420FD0DFF8F81188420BD0DFF8B7
S1131320F411884207D0DFF8F011884203D0DFF8C7
S1131330EC11884201D1012070470020704770B53C
S113134006460C461546FFF7AFFF002804D1E421FA
S1131350DFF8CC01FFF780F9002D08D0012D06D06D
S1131360022D04D0E621DFF8B801FFF775F906F580
S113137080602946C907016801D5214300E0A143E3
S1131380016006F58460A907016801D5214300E0E6
S1131390A143016070BDF8B504460D4616461F46CC
S11313A0FFF782FF002805D14FF4DD71DFF87001EB
S11313B0FFF752F9012E0BD0022E09D0042E07D0CC
S11313C00C2E05D04FF4DF71DFF85401FFF744F918
S11313D0082F11D00A2F0FD00C2F0DD0092F0BD0AE
S11313E00B2F09D00D2F07D0002F05D040F2C511C7
S11313F0DFF82C01FFF730F904F5A0603146C90786
S1131400016801D5294300E0A943016004F20450B6
S113141031468907016801D5294300E0A9430160E9
S113142004F5A16031464907016801D5294300E06C
S1131430A943016004F5A3603107016801D529437C
S113144000E0A943016004F20C503946C907016861
S113145001D5294300E0A943016004F5A26039469F
S11314608907016801D5294300E0A943016004F21A
S1131470145039464907016801D5294300E0A943BE
S1131480016004F21C5039460907016801D529435B
S113149000E0A943016004F5A560002F016801D1B3
S11314A0294300E0A9430160F1BD38B504460D4667
S11314B0FFF7FAFE002804D140F21F511848FFF745
S11314C0CBF8022229462046FFF739FF08230122E0
S11314D02946204601B0BDE830405CE70080054065
S11314E000500040009005400060004000A005400E
S11314F00070004000B005400040024000C00540BC
S11315000050024000D005400060024000E0054069
S11315100070024000F0054000D003400000064087
S1131520041800000746384600F022F8FBE7FF00E5
S113153080B50E480121017000F024F8BDE8014097
S113154010B5FFF779FA01280FD0084C207801284C
S11315500BD100F036F8322807D30020207000F0B9
S113156020F8BDE81040FFF769BA10BDE60400207A
S113157080B5C046C046024A11001820ABBEFBE746
S11315802600020080B500F00CF811484CF24F31EF
S1131590416000218160052101600020BDE8024016
S11315A00CE00B4800210160704709480068C00343
S11315B003D508480188491C018070470549088003
S11315C0704780B5FFF7F1FF0248008802BD0000B4
S11315D010E000E0E404002010E00F4014E00F40AD
S11315E01CE00F4010E00F4040E00F4044E00F408B
S11315F048E00F4000E10F4004E10F4008E10F40D4
S113160010E10F4014E10F4018E10F4020E10F40BA
S113161024E10F4028E10F4040420F0000201C004D
S113162080841E0000802500999E3600004038000A
S113163000093D0000803E0000004B00404B4C0080
S113164000204E00808D5B0000C05D0000807000B3
S113165000127A0000007D0080969800001BB700FD
S11316600080BB00C0E8CE00647ADA000024F400F5
S11316700000FA00443A5C7573725C6665617365D8
S1131680725C736F6674776172655C4F70656E42ED
S11316904C545C5461726765745C44656D6F5C4165
S11316A0524D434D335F4C4D33535F454B5F4C4D6F
S11316B03353383936325F4941525C426F6F745C40
S11316C06C69625C6472697665726C69625C737978
S11316D07363746C2E63000000200000002000007F
S11316E00100000000400000002000000200000093
S11316F000600000002000000300000000800000E3
S1131700002000000400000000A0000000200000F1
S11317100500000000C000000020000006000000DA
S113172000E00000002000000700000000000100AD
S1131730002000000800000000200100002000003C
S11317400900000000400100002000000A00000021
S113175000600100002000000B0000000080010078
S1131760002000000C00000000A001000020000088
S11317700D00000000C00100002000000E00000069
S113178000E00100002000000F0000000000020043
S113179000800000100000000080020000800000B3
S11317A0110000000000030000800000120000008F
S11317B0008003000080000013000000004000408F
S11317C0008005400050004000900540006000404B
S11317D000A005400070004000B0054000400240F9
S11317E000C005400050024000D0054000600240A7
S11317F000E005400070024000F0054000D00340C6
S113180000000640443A5C7573725C6665617365FA
S1131810725C736F6674776172655C4F70656E425B
S11318204C545C5461726765745C44656D6F5C41D3
S1131830524D434D335F4C4D33535F454B5F4C4DDD
S11318403353383936325F4941525C426F6F745CAE
S11318506C69625C6472697665726C69625C6770FB
S1131860696F2E630000000034E10F4004E40F4070
S113187008E40F400CE40F4030E10F4004E20F4055
S113188008E20F400CE20F40443A5C7573725C66E8
S113189065617365725C736F6674776172655C4FC2
S11318A070656E424C545C5461726765745C446547
S11318B06D6F5C41524D434D335F4C4D33535F4527
S11318C04B5F4C4D3353383936325F4941525C4299
S11318D06F6F745C6C69625C6472697665726C6962
S11318E0625C666C6173686C69622E630000000060
S11318F0443A5C7573725C6665617365725C736FA0
S11319006674776172655C4F70656E424C545C54CA
S113191061726765745C44656D6F5C41524D434D03
S1131920335F4C4D33535F454B5F4C4D3353383924
S113193036325F4941525C426F6F745C6C69625C21
S11319406472697665726C69625C756172746C69E3
S1131950622E6300443A5C7573725C6665617365FC
S1131960725C736F6674776172655C4F70656E420A
S11319704C545C5461726765745C536F7572636533
S11319805C41524D434D335F4C4D33535C4941529E
S11319905C766563746F72732E630000443A5C7501
S11319A073725C6665617365725C736F667477618C
S11319B072655C4F70656E424C545C54617267652D
S11319C0745C536F757263655C41524D434D335F74
S11319D04C4D33535C756172742E63002FF7FFFF17
S11319E0E80400000000002000000000402101483D
S11319F0FEF732BE54190000C046C046C046C04679
S10F1A00FFF778FB4F70656E424C5400F9
S90319F9EA
